:020000020000FC
:040000000DC031C23C
:0C000A00639519F4239409F42A941895C6
:10001A00F3C22FED2DBF2FEF27BB23E521BB23E032
:10002A002ABB25D220E828B920E02CBB22E020BF39
:10003A0024E023BF2DE426BF20E02FBD27E02EBDFC
:10004A0021E829BF71E090E0332444245524320189
:10005A00222720936000209361002093620019D325
:10006A0078948895FDCF2CE222BB903059F4222750
:10007A000CE2182D1F71103011F42FE70DE228BB86
:10008A0002BB0895983008F04FC0943008F081C040
:10009A00092F033008F001E0080F102F933011F4F4
:1000AA0084FC1127713031F0723081F07330D1F055
:1000BA00743021F1292D053008F02AE09FD0143040
:1000CA0009F4205828BB2DE222BB08952A2D0530B9
:1000DA0008F02AE093D0133009F4205828BB2EE206
:1000EA0022BB08952B2D053008F02AE087D0123064
:1000FA0009F4205828BB2CE322BB08952C2D053087
:10010A0028F0933011F42AE084FC2BE0203021F40B
:10011A00013011F02FEF04C071D0113009F42058CA
:10012A0028BB2CE622BB0895713031F0723079F089
:10013A007330C9F0743011F1209163005FD09830A8
:10014A0011F484FC2FEF28BB2DE222BB08952091E5
:10015A00640054D0993011F484FC2FEF205828BB46
:10016A002EE222BB08952091650048D09A3011F4FE
:10017A0084FC2FEF28BB2CE322BB08952091660054
:10018A003DD09B3011F484FC2FEF28BB2CE622BB18
:10019A000895713031F0723079F07330C1F07430F3
:1001AA0011F1209167002AD0943011F484FC2FEFCA
:1001BA0028BB2DE222BB0895209168001FD09530FC
:1001CA0011F484FC2FEF28BB2EE222BB0895209164
:1001DA00690014D0963011F484FC2FEF205828BB04
:1001EA002CE322BB089520916A0008D0973011F4BD
:1001FA0084FC2FEF28BB2CE622BB08952C3038F460
:10020A00F7E0EEE4E20F2227F21F249108952FEB84
:10021A000895A22D562F3CB54DB566276DBD6CBD10
:10022A0022245DD288279924AA24BB24650175015A
:10023A00303826E9420728E9520720E0A20718F0D9
:10024A0086E0D89A02C0AAD0E1D0933091F42FD098
:10025A0088279924AA24BB2465017501303826E928
:10026A00420728E9520720E0A20710F086E001C001
:10027A0095D02227F21629F4E21619F4D21609F4B7
:10028A0009C09A2CAB2CBC2CCD2CDE2CEF2CFF24D5
:10029A008395EFCF0895330C441C551C661C771CBC
:1002AA0028F477247A94672C2301372C0895332D68
:1002BA00A201D301309270004092710050927200F4
:1002CA006092730070927400E3E6F0E0D4E011C02B
:1002DA00E2DF232D82010301DEDFDDDF320E401E65
:1002EA00511E601C711C28F477247A94672C230110
:1002FA00372CC191C03041F0330D441D551DA61D48
:10030A00B71D28F0CA95C1F7DA9511F702C05FEF59
:10031A003AC0242F352FAD01AA27BB27220F331F3E
:10032A00441F551FAA1F232F8A010D01C3E01694EB
:10033A000794179507952795CA95C9F7321B400B5D
:10034A00510BA009B109C2E01694079417950795B5
:10035A002795CA95C9F7320F401F511FA01DB11D1D
:10036A00C3E016940794179507952795CA95C9F778
:10037A00320F401F511FA01DB11DA03019F4B0301B
:10038A0009F401C05FEF3090700040907100509006
:10039A00720060907300709074000895303422E403
:1003AA0042072FE0520728F0305442445F40F3944A
:1003BA00F5CF303A26E8420721E0520728F0305AB2
:1003CA0046485140E394F5CF303127E2420720E016
:1003DA00520728F0305147425040D394F5CF383E67
:1003EA0023E0420720F0385E4340C394F8CF343606
:1003FA0020E0420720F034564040B394F8CF3A3018
:10040A0018F03A50A394FBCF932E0895913089F4B3
:10041A0020916700A21620916800B2062091690017
:10042A00C20620916A00D2062227E206F206A0F04E
:10043A0011C020916700921620916800A2062091AF
:10044A006900B20620916A00C2062227D206E20695
:10045A00F20610F0D89A0895D898089520E225BF98
:10046A0020E02BBF91E022E02BBB82D0189520E33D
:10047A0025BF20E42BBF222728BB2BBB2CE222BBA3
:10048A000895943008F04AD19A959F3F09F493E071
:10049A0000D1933009F4DBDE0895E8E5F2E0E90FD4
:1004AA002227F21F09940BC00CC00BC00CC00EC04F
:1004BA0016C01EC026C02EC036C03EC046C0D7DFFA
:1004CA000895E7D00895E5D0C2DE08952091670027
:1004DA0023952A3008F02227209367000895209157
:1004EA00680023952A3008F022272093680008958F
:1004FA002091690023952A3008F022272093690069
:10050A00089520916A0023952A3008F02227209323
:10051A006A0008952091630023952A3008F0222763
:10052A002093630008952091640023952A3008F0EF
:10053A0022272093640008952091650023952A308C
:10054A0008F02227209365000895209166002395DC
:10055A002A3008F0222720936600089597E008952C
:10056A00772466242301332472DE08959BE00895DC
:10057A0020916100203019F02A95209361000091A2
:10058A00600020B32C7020936000021761F0009184
:10059A006100003041F422FF03C023FF03C003C0FF
:1005AA0070DF01C07ADF05E022FF0093610023FFBC
:1005BA0000936100233029F00091620003950093B3
:1005CA00620000916100003019F400E000936200BB
:1005DA0000916200063979F400E00093620020304D
:1005EA0049F022FF03C023FF03C005C0B7DF03C0E1
:1005FA00B7DF01C0BBDF089536DD7A9521F474E0D8
:10060A0003D0B6DF83941895913049F420916F0096
:10061A002A9520936F00E1F52AE020936F0020913C
:10062A006B002A9520936B002F3F91F529E02093C8
:10063A006B0020916C002A9520936C002F3F41F5A6
:10064A0029E020936C0020916D002A9520936D007B
:10065A002F3FF1F429E020936D0020916E002A9536
:10066A0020936E002F3FA1F42091630020936B002A
:10067A002091640020936C002091650020936D0006
:10068A002091660020936E002AE020936F00C1DD5E
:10069A0008952FEF922EA22EB22E65017501209198
:1006AA00630020936B002091640020936C002091DA
:1006BA00650020936D002091660020936E002AE069
:1006CA0020936F00A22D562F3CB54DB566276DBD00
:1006DA006CBD222404D0882710D0BEDE08952FEFE7
:1006EA00721639F02227330E441E551E6A1E721ED8
:1006FA0008F008952FEF722E0895F894E199FECF2D
:10070A000027E3E6F0E00EBBE09A2DB32A3008F0AA
:10071A0020E0219303950830B0F30895F894112747
:10072A00E3E6F0E0E199FECF1EBBE09A2DB301911A
:10073A00201721F01EBB0DBBE29AE19A13951830DF
:10074A0088F30895C0F9A4B0999282F88090FF8640
:00000001FF
